:1000000044C200005EC200005CC200000C945A0FA3
:1000100058C2000056C2000054C2000052C2000084
:1000200050C200004EC200000C94EE264AC20000EE
:1000300048C2000046C2000044C2000042C20000A4
:1000400040C200000C949B103CC200003AC2000069
:1000500038C200005FC5000034C2000032C2000098
:1000600030C200002EC200002CC200002AC20000D4
:1000700028C2000026C2000024C2000022C20000E4
:1000800020C200001EC200001CC200001AC20000F4
:1000900018C2000016C2000014C2000012C2000004
:1000A00010C200000EC200000CC20000425A0862DA
:1000B0000A28433B03461F0C699E1B4155175AD023
:1000C0001945D01A47650A4D210B4B9D0A55360A32
:1000D00059D01C52090854E02056E10757D108585E
:1000E000861365900866AE226D9D236C8108742985
:1000F0000675191578630400000012011001020052
:100100000008EB034B20000001020001090243003C
:1001100002010080320904000001020201000524EE
:100120000001100524010301042402060524060031
:1001300001070582030800FF09040100020A00000C
:100140000007050402400000070583024000000488
:1001500003090416036200750073007700610072E2
:100160000065002E006400650000002A034300556E
:10017000004C0038003600380000002A03430055C8
:10018000004C00340033003300000000030F1E2633
:1001900027000000030F1E2536386700030F256770
:1001A00040605000030F275188838100030F2750C0
:1001B000C8C3C20027000000000000006700000064
:1001C000000000005000000000000000810000005E
:1001D00000000000C20000000000000D2E2D07D31B
:1001E000913D04320000060021656A55E43023B9D0
:1001F00000070018146C070090876BF85611E92A65
:10020000001F4100072E050DD391FF080500000CCB
:100210000021656A2D3B1322F862073F181D1CC799
:1002200000B0876BF8B611EA2A001F4100202F208A
:1002300000203D2000504C4C310D0A00504C4C30F9
:100240000D0A005620312E36312043554C383638B1
:10025000005620312E36312043554C343333004381
:10026000554C5F563300202F2000203D20004C4F7E
:1002700056460D0A00424F56460D0A000007022E50
:10028000030D04E905CA070C0B060D210E650F6A64
:1002900010C81193120315341733181819161B437D
:1002A00021562500261129592C812D353EC30B08D6
:1002B000105B11F81547191D1A1C1BC71C001DB235
:1002C00021B623EA0007024604C605260B0610C81D
:1002D0001193120313221534173F182819161B43C4
:1002E0002156250026110D210E650F6A070C1607F1
:1002F00020F81E871F6B29592C812D353EC3FF0026
:100300004C454E4552520D0A004C4F56460D0A00C0
:100310004C454E4552520D0A0000070246030D049B
:100320009A057D0642070C0B060D210E650F6A101B
:10033000C81193120315341700181819161B431C03
:100340006825002611FF00000000000000000000EA
:1003500000000000000D2E2D07D3913D0432000057
:10036000060010B07155E43023B900070018146C72
:10037000070090876BF85611E92A001F41000D2EE7
:100380002D07D3913D04320000060010ABA5550A9D
:100390003023B900070018146C070090876BF856DB
:1003A00011E92A001F410000535300547D7DFFFFD7
:1003B0004B4B7E7E00454F420D0A004E2F41004EB2
:1003C0002F410020697320756E6B6E6F776E292048
:1003D000557365206F6E65206F66003F202800040E
:1003E0007605961700000602000B080C000D210E82
:1003F000650F6A106A114A1206132214F80A0015D2
:100400004721B622101818192E1A6D1B041C091D3D
:10041000B223EA242A2500261F29592C812D352EA6
:100420000907000800090006FF3EC2FF0454053D0D
:100430001700000602000B080C000D210E6B0FD0F8
:10044000105C11041206132214F80A00154421B698
:1004500022101818192E1ABF1B431C091DB523EAB8
:10046000242A2500261F29592C812D352E09070005
:100470000800090006FF3EC2FF4F464600544D4F9C
:10048000444500534D4F4445000011241FBECFEF9B
:10049000DAE0DEBFCDBF11E0A0E0B1E0E6E2FAE5D0
:1004A00002C005900D92AE38B107D9F718E0AEE85A
:1004B000B1E001C01D92A63DB107E1F70CD00C944C
:1004C000112D9ECDF89481E085BF82E085BFE0E0EC
:1004D000F8E3099508952FE088E190E00FB6F894CD
:1004E000A895809360000FBE2093600080E090E0AC
:1004F00020E80FB6F89420936100809361000FBE4E
:100500002E9A2D9A04B603FE0AC083E390E069D5C3
:10051000882329F083E390E060E0C7D5D3DF89EF3B
:1005200087BD84E085BD82E084BD80936E0010921B
:1005300080008AE08093810084B7877F84BF6E9AB1
:100540000E9469231BD60E94D5260E94BF200E94CC
:10055000220C86E293E290938E0380938D030E9497
:10056000BB1589E08093930176980E949E270DD257
:100570000E94091111D30E9449220E94A0130E94D7
:10058000CE150E9457190E94181A0E949A28EDCF82
:10059000DA01292F33272230310559F02330310574
:1005A00069F02130310561F54AEF50E022E130E099
:1005B0002BC04CE051E023E430E026C09070813045
:1005C000910551F08130910518F00297C9F40BC0E4
:1005D000EFE4F1E0849103C0E3E5F1E08491282F9A
:1005E00030E0AF0111C01E9B03C04BE651E002C0DA
:1005F0004BE751E0EBE6F1E0E4912E2F30E004C050
:1006000040E050E020E030E04D935C93C901089554
:100610008EBD0DB407FEFDCF8EB508952898806C71
:100620008EBD0DB407FEFDCF8EB51EBC0DB407FE0A
:10063000FDCF8EB5289A0895289880648EBD0DB49C
:1006400007FEFDCF8EB56EBD0DB407FEFDCF8EB596
:10065000289A089528988EBD0DB407FEFDCF8EB55B
:10066000289A089586E3F6DF10928F0310923C02D9
:1006700010923E020895A1E0B0E0E1E4F3E00C94B2
:10068000CD2B0196BE016F5F7F4F41E036D4892BA1
:1006900041F18981893989F400E010E0802FBEDFC3
:1006A000EBD3C80187709070079709F493D30F5F5D
:1006B0001F4F0033110591F714C0B0DF182F83E4EA
:1006C00054D38981D9D381E392E088D3812FD4D3C5
:1006D0008DE292E083D3812F90E062E040E2D0D3BC
:1006E00079D32196E4E00C94E92B1F931FEF05C00A
:1006F0008AE090E0BBD2112331F084E3ABDF1150EC
:1007000080778031A9F7EA9A1F9108951F93EA989C
:1007100086E3A0DF1FEF05C08AE090E0A7D2112397
:1007200031F085E397DF115080778032A9F71F9170
:100730000895EF92FF920F93CF93DF93082F8A30A3
:1007400008F008E0C02FD0E083E0CC0FDD1F8A95D1
:10075000E1F7C557DE4F8BE290E07C010894E11C85
:10076000F11CFE016491A1D42196C7018333910548
:10077000A1F70550053010F067E101C061E184E2A6
:1007800090E093D4DF91CF910F91FF90EF90089577
:10079000CF93DF9382E090E0EC012196FE01E852D6
:1007A000FE4FE4916E2F81D4CB32D10511F0CE01F2
:1007B000F3CF87E390E0EC012196FE01E453FE4F76
:1007C000E4916E2F72D4C036D10511F0CE01F3CF73
:1007D0001E9918C08FE090E060E167D480E190E05E
:1007E00060EB63D481E190E061E75FD484E490E062
:1007F00060E15BD485E490E060EB57D486E490E060
:1008000061E753D488E095DFDF91CF9108950F938E
:100810001F93CF93DF938C0110923E02EA98209AA7
:10082000289A8EE190E022D228988EE190E01ED2A4
:10083000289A8DE290E01AD280E30CDF84E690E003
:1008400015D2289880E48EBD0DB407FEFDCF8EB57D
:10085000C0E0D0E0C8018C0F9D1FC3D38EBD0DB486
:1008600007FEFDCF8EB52196C932D10599F7289A9A
:1008700028988EE78EBD0DB407FEFDCF8EB58BE2B6
:1008800090E0EC012196ADD38EBD0DB407FEFDCFF7
:100890008EB5C333D10511F0CE01F3CF289A83E38F
:1008A000D9DE81E0E8D1DF91CF911F910F910895BA
:1008B00082E090E0ACDF81E080938F0310923C02F5
:1008C00010923E020895A1E0B0E0E9E6F4E00C9455
:1008D000CF2B22E029830196BE016F5F7F4F41E05D
:1008E0000CD3898126DF82E090E091DF2196E2E05F
:1008F0000C94EB2BFF920F931F93F82E062F1FEFF4
:1009000085E38CDE8F1549F0802F90E0AFD1112365
:1009100011F481E003C01150F3CF80E01F910F91DB
:10092000FF90089585E27ADE8F33F1F486E392DE5C
:1009300080918E01882321F48CE392E04FD202C093
:100940008DE388DE83E386DE81E064E0D3DF85E249
:1009500065DE8F3349F480918E01882319F485E395
:1009600092E03CD281E0089580E0089585E356DE70
:100970008D3051F485E252DE8F3331F4D3DF84E3DE
:1009800069DE80778031D9F70895809152058430EF
:1009900009F069C08093E90080918F01882351F5A7
:1009A0008091E80085FD06C025C06091F1008BECC8
:1009B00094E045D48091F2009091F300892BA9F73F
:1009C0008091E800982F9B7F9093E8008F77809329
:1009D000E80081E080938F0185EC94E090938C0394
:1009E00080938B03E0918D03F0918E0381E0099554
:1009F00010928F0183E08093E90080914A0488235C
:100A000091F18091E80085FF2EC0F89405C088E43C
:100A100094E02DD48093F10080914A04882339F02A
:100A20008091F2009091F3008034910580F37894E6
:100A30008091F2009091F3002091E800322F3E7FE8
:100A40003093E8002F772093E8008034910559F423
:100A50000E9476258091E800982F9E7F9093E80071
:100A60008F778093E8000895909153058091540505
:100A7000813229F0823261F1803299F512C0913AC7
:100A800081F58091E800877F8093E80080E091E025
:100A900067E070E00E94A1258091E800982F9B7F7D
:100AA00011C09132F1F48091E800877F8093E800D3
:100AB00080E091E067E070E00E9443268091E800CA
:100AC000982F9E7F9093E8008F778093E800089599
:100AD000913239F48091E800877F8093E8000C948C
:100AE0004D25089582E061EC42E00E94232583E0D9
:100AF00061E842E30E94232584E060E842E30E942B
:100B0000232510920001109201011092020110920F
:100B1000030108951F920F920FB60F9211248F9325
:100B20009F93AF93BF938091910390919203A09173
:100B30009303B09194030196A11DB11D809391037D
:100B400090939203A0939303B093940380919003A6
:100B50008F5F80939003809190038D3710F01092F7
:100B600090038091330490913404009729F0019709
:100B70009093340480933304809146048F3F19F09E
:100B8000815080934604BF91AF919F918F910F90B8
:100B90000FBE0F901F901895809191039091920332
:100BA000A0919303B091940320919101281709F427
:100BB0004FC08091910390919203A0919303B091C3
:100BC000940380939101A89580913304909134040B
:100BD000892B11F40E945A2080914604882311F435
:100BE0000E94412080912304882339F08150809312
:100BF0002304882311F40E94FD148091900388231C
:100C000039F58091070181FF04C08EB190E48927F6
:100C10008EB9809195039091960323E084389207D2
:100C200028F4019690939603809395038091900108
:100C30008F5F809390018C3359F4109290018091D2
:100C400030048F5F809330048C3310F010923004A6
:100C500008958091940310D1809193030DD18091D8
:100C600092030AD18091910307D1B4C0880F991FD4
:100C70000197F1F7089520ED37E004C0F9013197AD
:100C8000F1F781508823D1F70895CF93DF93AC011A
:100C9000DC0113968C911397843509F063C09C9105
:100CA0002DE001C02F5F291730F4FA01E20FF11D8A
:100CB00083818B33B9F730E0E92FF0E0CF010F9754
:100CC0002817390709F04EC03E979A012E0F3F1F93
:100CD0003E96D90113968C91843509F043C03B9719
:100CE000EA01CE0FDF1F3B96DA0114969C91149710
:100CF00089819817B9F515969C9115978A8198174F
:100D000089F516969C9116978B81981759F5179629
:100D10009C918C81981731F57197E40FF51F8D81A7
:100D20008383F90131968E81D90111968C93DF016D
:100D3000119689858183FD0131968A8511968C9360
:100D4000DF0111968B8581838C8511968C93119789
:100D50008D8512968C93FA0180818A5080838281DE
:100D60008A508283DF91CF9108951F93182F80912D
:100D70005205843081F48091930180FF0CC08091F2
:100D80004A0487FF01C001DE88E494E0612F57D256
:100D90001A3009F4FADD80912E048823C9F080917D
:100DA000930183FF15C01A3099F01D3011F46BE3E5
:100DB00001C0612F8EE993E042D21D3019F48EE913
:100DC00093E063DF83E08093230482E0809329042F
:100DD0001F9108958DE0C9DF8AE0C7CFCF93DF93DD
:100DE000EC0102C0C2DF2196FE0184918823D1F775
:100DF000DF91CF910895CF93DF93EC0102C021964C
:100E0000B4DF88818823D9F7DF91CF910895A5E0D9
:100E1000B0E0EDE0F7E00C94CF2B1D8234E0DE0172
:100E20001196282F2F7031502A3010F4205D01C008
:100E3000295CFD01E30FF11D208324E09695879541
:100E40002A95E1F76150009761F706C03150FC0127
:100E5000E30FF11D408302C0CE010196615067FD92
:100E600002C0332399F7CE010196830F911DC3DF92
:100E70002596E2E00C94EB2B90E062E040E3C7CFD4
:100E8000A6E0B0E0E6E4F7E00C94CB2B9C01162F33
:100E9000042F1E8245E07E010894E11CF11C4150A4
:100EA000F701E40FF11DC9016AE070E00E94982B80
:100EB000805D8083C9016AE070E00E94982B9B01ED
:100EC00011506115710549F0442349F706C041509E
:100ED000FC01E40FF11D008302C0CE010196115008
:100EE00017FD02C0442399F7CE010196840F911D8E
:100EF00082DF2696E6E00C94E72BDC01FB0123C0A1
:100F0000822F80538A3010F050E002C0382B51E01D
:100F1000822F8154863020F42753322B295C51E0F4
:100F2000822F8156863018F42755322B07C055235F
:100F300029F4203271F02A3361F00EC0992331F088
:100F40003193415049F030E090E003C03295307F5A
:100F500091E02D912223A1F6CF01861B970B0895D6
:100F6000FC01DB0120E030E014C0842F80538A3084
:100F700080F4C90163E0880F991F6A95E1F7220F99
:100F8000331F820F931F242F30E020533040280F4F
:100F9000391F4191442349F72D933C930895FB0158
:100FA000982F92959F709A3010F4905D01C0995CD3
:100FB00090838F708A3010F4805D01C0895C8183DA
:100FC0000895FC018181883419F48FE592E007C00F
:100FD0001E9903C081E592E002C083E492E0FEDE48
:100FE000F9CE0C94FB2C08951F93CF93DF93EC0163
:100FF000162F09C01150CE01F4DF3EDF112311F08E
:101000008AE3B3DE21961123A9F7DF91CF911F91D7
:101010000895EF92FF921F93DF93CF9300D0CDB747
:10102000DEB7FC0181818D3421F48AEF93E066E024
:1010300005C0803529F48AED93E060E1D5DF2CC04E
:101040001A821982CF010196BE016F5F7F4F42E085
:1010500054DF2981823041F4922F80E02A81E22EF0
:10106000FF24E82AF92A02C0E22EFF24C701B9DFD3
:10107000182F82E57ADEC70164E040E3C8DE8AE625
:1010800092E0ACDE812FF8DE86E692E0A7DE812FCB
:1010900090E062E040E2F4DE9DDE0F900F90CF9191
:1010A000DF911F91FF90EF9008950E94032DF99911
:1010B000FECF0895A1E0B0E0E0E6F8E00C94CF2B7D
:1010C0001982009731F00196BE016F5F7F4F41E0BA
:1010D00014DF8981882321F083E390E061E0E5DF7C
:1010E0000E94C32610926E00F89428E088E190E0F8
:1010F0000FB6F894A895809360000FBE209360000F
:10110000FFCF019667E071E041E0F7DE60910701F3
:1011100060FF02C0769A01C0769884E390E0C5CF64
:101120000F931F938C0180E090E061E0BEDF81E0CF
:1011300090E06DE3BADF2CDB80E690E060E0B5DFA5
:1011400081E690E060E0B1DF83E390E060E0ADDF56
:1011500084E390E062E0A9DF80E690E060E0A5DF54
:1011600081E690E060E0A1DFF8018181883719F025
:1011700080E090E09FDF1F910F91089580E090E064
:1011800030DF813029F481E090E02BDF8D3319F0DE
:1011900080E090E0C5DF84E390E023DF80930701E7
:1011A0000895A6E0B0E0E7EDF8E00C94C92B6C01DF
:1011B0000196BE016F5F7F4F43E09FDE082F8230B4
:1011C000A8F12981823019F4E22EFF2407C0922F62
:1011D00080E02A81E22EFF24E82AF92A10E0FE01AD
:1011E000E00FF11FC701608160DF000F111F0F5F6B
:1011F0001F4F0C0D1D1D0894E11CF11C6E0108947D
:10120000C11CD11C0FC0C801B60141E076DE892B9C
:1012100069F0C701698149DF0E5F1F4F82E090E0EE
:10122000E80EF91EF8018081882369F72696E8E028
:101230000C94E52BFC011282108211820895DC01CE
:101240009FB7F89412968C91129787FD0EC08F5F0E
:1012500012968C9312978C91FD01E80FF11D638318
:101260008F5F8C93803809F41C929FBF0895DC0136
:101270002FB7F89412968C911297882319F42FBFE8
:1012800090E014C0815012968C93129711968C9115
:101290001197FD01E80FF11D93818F5F11968C93DB
:1012A0001197803811F411961C922FBF892F089541
:1012B000CF93DF93DB01EA01322F4881882369F065
:1012C000FB01E40FF11D81E090E002C0880F991F3F
:1012D0002A95E2F72081282B2083332319F0832FCE
:1012E000815009C0842F8F5F8C3008F48883A80F49
:1012F000B11D1C9287E090E0DF91CF9108951F937C
:10130000182F5B9A882319F08091960102C0809172
:10131000940190E034E0880F991F3A95E1F7A6DC3C
:101320005B98112319F08091970102C0809195017B
:1013300090E024E0880F991F2A95E1F797DC1F9130
:101340000895A0E0B0E0E7EAF9E00C94C12B4C016D
:10135000562ED42E122FC02E4E2C20919503309154
:10136000960382E0D80ED09E802D11249EEFD90ED8
:10137000992787FD90952817390720F48EE692E08B
:101380002DDD6FC0281B390B3093960320939503F6
:10139000769A80913E02882311F4EE2408C01092C0
:1013A0003E0288E091E00E948613EE24E39480914F
:1013B0008F03882309F47CDAA9D941E0642E712CCB
:1013C000A12EBB2410E003C080E099DF1F5F15153C
:1013D000D9F7552011F081E092DF8401FF2415C078
:1013E000C7E0D0E093010C2E02C0220F331F0A94F5
:1013F000E2F7F8018081822382DF2197FFEFCF3F60
:10140000DF0781F7F3940F5F1F4FFD1449F7C7E023
:10141000D0E00D2D112707FD1095080D191D0CC0EA
:1014200093010C2E02C0220F331F0A94E2F7F80139
:101430008081822364DF2197AC16BD068CF3842D56
:101440001ADCCA9409F0BECF80919703882311F06B
:101450004CD902C086E3FED8EE2011F00E946D1731
:101460007698CDB7DEB7E0E10C94DD2BEF920F93C9
:101470001F93DF93CF9300D000D0CDB7DEB7019696
:101480008E010F5F1F4FB80143E037DD9AE690935E
:10149000940184E28093950181E280939601909378
:1014A000970180E88C83C80160E043E026E003E018
:1014B0005FE0E52E46DF0F900F900F900F90CF91D9
:1014C000DF911F910F91EF900895EF920F93DF93AB
:1014D000CF93CDB7DEB760970FB6F894DEBF0FBEDF
:1014E000CDBF0196BE016F5F7F4F40E106DD698190
:1014F0004A810B818C81809394018D818093950129
:101500008E81809396018F8180939701242F2F7075
:10151000E02EE2947FE0E722CE01089642954F70DC
:101520000F700FDF60960FB6F894DEBF0FBECDBF11
:10153000CF91DF910F91EF900895A9E1B0E0E3EA38
:10154000FAE00C94BF2B8E01025F1F4F0196B80189
:101550004BE0D3DCF82E95E39093940186E18093E1
:1015600095018093960190939701C8016F2D9AD1B0
:10157000F801EF0DF11D80836F2C639419821A829C
:101580007724E7E0A1E02A2E312C2801F2E08F2E0B
:10159000912C8C0E9D1E5E010894A11CB11C41C0B3
:1015A00000E010E0C72CDD247201EC0CFD1C910161
:1015B000002E02C0220F331F0A94E2F7D7018C914C
:1015C0008223B401A5012E2F73DEE82F0F5F1F4F7A
:1015D0000430110561F781E0B401A5012E2F68DE0A
:1015E000982F04E010E07201EC0CFD1C9101002E1C
:1015F00002C0220F331F0A94E2F7F7018081822391
:10160000B401A501292F54DE982F0F5F1F4F08301A
:10161000110561F781E0B401A501292F49DEE82F0A
:101620007394761408F4BCCFCE0102966AE0498127
:101630002E2F03E0EAE0EE2E84DE6996E2E10C94C0
:10164000DB2BA9E1B0E0E7E2FBE00C94C32B3EE02A
:10165000E32EF12CEC0EFD1E0196B7014BE04DDCA4
:10166000893009F05BC089E18093950180939401F2
:101670008093960182E380939701C70169E005D1C9
:101680008F8B19821A8207E0A7E010E027E0622E14
:10169000712C91E0892E912C570182E0C82ED12C1B
:1016A000CC0EDD1E7E010894E11CF11C01C007E098
:1016B000802F992787FD90959301281B390BC40132
:1016C00002C0880F991F2A95E2F79C01F501E10FEE
:1016D000F11D80818223B601A7012A2FE9DDA82F01
:1016E000002311F00150E4CF81E0B601A7012A2FB9
:1016F000DFDDA82F1F5F1A30D0F2882319F0282FC2
:10170000215004C089818F5F898327E0CE01029632
:101710006CE0498103E0BAE0EB2E13DE6996EEE05F
:101720000C94DF2BAEE0B0E0E8E9FBE00C94BF2BBB
:101730007C01162F842F2E87B701412F9AD0F701F5
:10174000E10FF11D8083A12EA39419821A82470113
:10175000BB24E7E0F1E02F2E312C72E0472E512C14
:101760004C0E5D1E3E010894611C711C2FC007E0E9
:1017700010E06701CB0CD11C9101002E02C0220F9A
:10178000331F0A94E2F7D6018C918223B201A301A0
:101790002E2F8EDDE82F01501040BFEF0F3F1B07AB
:1017A00059F7D4018D914D01082E82958025082E80
:1017B00086958695802590E0019695958795817010
:1017C000B201A3012E2F74DDE82FB394BA1478F27E
:1017D000EE2319F02E2F215004C089818F5F898359
:1017E00027E089E1809395018093940185E28093BD
:1017F000970180939601CE0102966CE049810E8597
:101800005AE0E52E9EDD2E96E2E10C94DB2BACE057
:10181000B0E0EDE0FCE00C94CB2BF62EE42E01962C
:101820008E010F5F1F4FB8014BE067DB682FC801C7
:101830004F2D2E2D77DF2C96E6E00C94E72B66E0FB
:1018400043E0E5CF539A5B985298E9E6F0E0808157
:101850008061808382EC91E090939603809395035E
:101860001092B4011092D0011092EC0110928F03EB
:101870000895982F06C04150FB01E40FF11D8081AF
:10188000980F4423C1F7892F0895AC0120E006C0CA
:101890006150FA01E60FF11D808128276623C1F708
:1018A000822F0895DC019091200230E025E040E095
:1018B00013C06150FD01E60FF11DE0818E2F82956E
:1018C0008F703827280F992311F0442321F08E2F91
:1018D0008F703827280F4F5F662359F7230F229503
:1018E000207F822F832B0895A0E0B0E0EAE7FCE0A0
:1018F0000C94C92BDC011092200210920B0297E08D
:1019000013968C911397981B11961C911197110F98
:10191000110F110F190F10920C02FF24EE2407E093
:1019200057E040E070E0E7E0CE2ED12CC1E0D0E0FF
:101930007FC0FD01EE0DF11D848190E0002E02C0FC
:10194000959587950A94E2F7282F2170002311F0CE
:10195000015002C0E39407E06B3469F4533059F44A
:101960007723B9F5222311F071E062C040930B0296
:10197000109220021EC05F3F69F56634E1F4E42F47
:10198000F0E0E45FFD4F8081082E82958025082ECF
:1019900086958695802590E001969595879581702E
:1019A000907030E08217930761F040930B027093C0
:1019B000200280E057C0653411F06B3411F422230B
:1019C000A1F34F5FE42FF0E0E45FFD4F108257E09A
:1019D0002FC070E0222359F1663479F4E42FF0E04F
:1019E000E45FFD4F9E01052E02C0220F331F0A94B3
:1019F000E2F78081822B80831AC0653411F06B344A
:101A0000B1F4E42FF0E0E45FFD4F852F992787FDC7
:101A100090959601281B390BC9019E0102C0220F27
:101A2000331F8A95E2F7C9012081282B208351506A
:101A3000F3948F2D8150811708F47BCF40930B02D4
:101A4000709320021F1508F0B4CF653411F45F3F86
:101A500011F0772319F04F5F40930B0280910B0236
:101A6000811181E0CDB7DEB7E8E00C94E52BDC0115
:101A700012968C911297ED91FC911197E80FF11D40
:101A8000E08113962C911397215013962C93139762
:101A90002F5F39F48F5F12968C93129787E013961D
:101AA0008C938E2F90E002C0959587952A95E2F74A
:101AB00081700895A0E0B0E0E0E6FDE00C94C52B55
:101AC0006C01962E842EFF24C0E0D0E0F1E0AF2E12
:101AD000B12C062F10E00150104019C0C601C7DF1D
:101AE0008823A1F0882059F0C8018C1B9D0B95011B
:101AF00002C0220F331F8A95E2F7C90106C0C50153
:101B000002C0880F991FEA94E2F7F82A2196EC2E7A
:101B1000C91520F38F2DCDB7DEB7ECE00C94E12B87
:101B2000A4E0B0E0E6E9FDE00C94C72BFC0187E0FF
:101B30008C833496FA83E983349710920B02818167
:101B400090E023E0880F991F2A95E1F72381821BFB
:101B50009109CE970CF45AC01B82CC24DD245E017F
:101B60000894A11CB11C2EC0ED2CFF24C50168E017
:101B700040E0A0DF082F8CE092E0E80EF91EF701AC
:101B80000083002E02950025002E0695069500255F
:101B9000C5016DDF10E00F5F1F4F159507950170B0
:101BA000107090E00817190731F4C50160DF9D2D12
:101BB0009F5F882319F0D0920B0228C0F701808123
:101BC000C826D92EF5E0FD1578F6D0920B02C50196
:101BD00068E040E06FDFF82E082F002E0295002508
:101BE000002E069506950025C50141DF10E00F5F28
:101BF0001F4F159507950170107090E00817190791
:101C000029F480E0CF1419F481E001C080E024962B
:101C1000EAE00C94E32BA4E0B0E0E1E1FEE00C94F8
:101C2000C72BFC011B8287E08C833496FA83E983FF
:101C3000349710920B028081853009F053C0818166
:101C400090E043E0880F991F4A95E1F72381821BBA
:101C500091098938910509F045C019E83FE0C32E84
:101C600030EFD32E80E05E010894A11CB11C10C09F
:101C7000C50168E041E01EDFC80ED11C2CE032E057
:101C8000E20EF31E1827F7011083182F1C5D802F1A
:101C9000E82EFF24082F0F5F8F3050F3C50168E056
:101CA00041E008DF182F2CE032E0E20EF31E8095B1
:101CB000F701808300930B02C50168E041E0FADE82
:101CC000082FC10ED11CC50168E041E0F3DE40E001
:101CD000302F20E0C21AD30A90E0C816D90619F4B2
:101CE00041E001C040E0842F2496EAE00C94E32B0D
:101CF000EF92FF921F93DF93CF9300D000D0CDB728
:101D0000DEB7FC013496FA83E9833497818184300D
:101D1000B9F587E08C838381813091F51B8210E0D7
:101D20007E010894E11CF11C12C0112331F4C7019B
:101D300067E041E0BFDE806804C0C70168E041E0C1
:101D4000B9DEE12FF0E0E45FFD4F80831F5F1430C8
:101D500060F3CE01019667E041E0ACDEE12FF0E0F8
:101D6000E45FFD4F880F80831F5F10930B0290E0AC
:101D700080910C0282958F708A3019F491E001C035
:101D800090E0892F0F900F900F900F90CF91DF91DF
:101D90001F91FF90EF900895FC018181A82FB0E082
:101DA00050E0E081CD01841B950B0B964797D8F44A
:101DB0008E2F90E070E09C01261B370B2C303105F4
:101DC00094F4255F3F4F7CF08A0F9B1F861B970B77
:101DD000841B950B8C30910534F420E0855F9F4F78
:101DE0001CF021E001C020E0822F0895282F30E070
:101DF000C901880F991F820F931F860F911D95951A
:101E00008795959587950895DC0111968C9111978A
:101E1000843190F010926F008091080290E02CE1E4
:101E200030E0829FF001839FF00D929FF00D11240E
:101E3000E856FE4F10820895662381F0FD01E80FF9
:101E4000F11D81E090E013960C90139702C0880F6B
:101E5000991F0A94E2F72481282B248313968C91EE
:101E60001397815013968C9313978F5F79F487E0C3
:101E700013968C93139711968C9111978F5F1196EF
:101E80008C931197A80FB11D14961C920895282FBA
:101E90008552873160F46A3050F0673240F490E048
:101EA000621708F091E081E09827892F089580E07B
:101EB00090E008951F920F920FB60F921124EF92A7
:101EC000FF920F931F932F933F934F935F936F93C3
:101ED0007F938F939F93AF93BF93CF93DF93EF93B2
:101EE000FF9380914704882321F082E08093470488
:101EF000F0C080912404823021F483E08093240494
:101F0000E8C08091840090918500E4E096958795E3
:101F1000EA95E1F7182FE09008028CE1E89EE001D5
:101F20001124C856DE4F9881943031F41E3208F4E3
:101F3000D0C01F3448F0BDC0953031F4173108F4DB
:101F4000C8C0183208F0B5C0892F84504A990CC017
:101F5000823038F4CE0161E057DF10928500109294
:101F6000840010933A02B5C000913A02F12EF01AA3
:101F7000F0923B021092850010928400823020F48F
:101F8000CE0160E041DFA5C082E086BB992371F4F9
:101F9000053608F09EC084E68F1508F49AC0088FB5
:101FA000F98E81E08A8382E0888393C0923009F0C1
:101FB0005AC0CE014896602F4F2DEEDE1A8188233D
:101FC00059F0888D602F12DF888F898D6F2D0EDF7D
:101FD000898F1F5F1A837DC0143008F442C080EAE5
:101FE0009FE090938900809388001C3050F0298DE9
:101FF000888D90E0820F911D8536910514F084E064
:1020000025C01A3080F0298D888D90E0820F911DB7
:1020100085974CF485E0888388EE93E0909389005F
:102020008093880014C080919D03882371F0802FD5
:102030006F2D2DDF882349F0898D688D28DF882357
:1020400021F081E08093240434C083E088830A8FE8
:10205000FB8E198287E08B831C8282E080936F0065
:1020600038C0188295CFCE014A96602F4F2D94DE4E
:10207000882361F0CE0161E0C7DE8A8D602FB6DE75
:102080008A8F8B8D6F2DB2DE8B8F23C0CE01489649
:10209000602F4F2D81DE882361F0CE0160E0B4DE39
:1020A000888D602FA3DE888F898D6F2D9FDE898FAD
:1020B00010C010926F002E2D30E08CE190E0289F30
:1020C000F001299FF00D389FF00D1124E856FE4FC6
:1020D0001082FF91EF91DF91CF91BF91AF919F91CE
:1020E0008F917F916F915F914F913F912F911F91B0
:1020F0000F91FF90EF900F900FBE0F901F901895CB
:102100008091080290E02CE130E0829FF001839FF3
:10211000F00D929FF00D1124E856FE4F8081882328
:1021200031F420E030E0809146048F3F11F021E04F
:1021300030E0822F08951F920F920FB60F92112454
:102140002F933F934F935F936F937F938F939F93BF
:10215000AF93BF93EF93FF9310926F00809197031B
:1021600083FF03C08EE20E94B50640910802242F2F
:1021700030E08CE190E0289FF001299FF00D389F1E
:10218000F00D1124E856FE4F8081833018F08181D4
:10219000823028F410926F008CE190E013C080919F
:1021A0000A028330D1F48091970382FF04C085E74F
:1021B00092E00E94EE0610926F008091080290E07B
:1021C0002CE130E0829FF001839FF00D929FF00D93
:1021D0001124E856FE4F10820BC08F5F80930A02D5
:1021E000842F8F5F80930802843011F410920802CC
:1021F000FF91EF91BF91AF919F918F917F916F91DF
:102200005F914F913F912F910F900FBE0F901F90B4
:1022100018950F931F93CF93DF9380913B028823F0
:10222000B9F18091970387FF17C084E30E940E03E2
:102230008058803410F480E00CC0803C10F08FE0B7
:1022400008C090E08055904003E0959587950A95E9
:10225000E1F78F590E94B5068091970383FF16C05E
:1022600082E70E94B5068091970384FF04C08091A5
:102270003A020E94B50686E60E94B5068091970351
:1022800084FF04C080913B020E94B50610923B027D
:1022900080910A02882309F42AC2769A9091090251
:1022A0008CE1989FE0011124C856DE4FCE01B3DCCB
:1022B000882311F003E5A8C0CE0166E415DB88236E
:1022C00009F4ECC140910B02415040930B02942F52
:1022D00056E007C09150E92FF0E0E45FFD4F8081A8
:1022E000580F9923B9F7A42FB0E0FD01E45FFD4F2B
:1022F0006081561711F4443068F4852F90E0019600
:10230000262F30E08217930779F4443068F0A45FF9
:10231000BD4F5C9306E478C09150E92FF0E0E45F94
:10232000FD4F8081280F02C0942F2CE09923A1F744
:10233000261709F0B3C1443008F4B0C1ADC1809193
:102340000B02815080930B02893009F0ADC199E0F6
:1023500020E09150E92FF0E0E45FFD4F80812827D5
:102360009923B9F780911502281709F09DC105E45A
:102370004BC060910B02615060930B028CE092E0C5
:1023800091DAE0910B02F0E090912002E91BF10953
:10239000E45FFD4F9081891761F08B818F5F8B83A4
:1023A0008150873009F09EC11B82898181508983C9
:1023B00099C10BE429C08B81843009F0E4C0CE01BF
:1023C00048966CE34EE1E8DC882309F4DCC0C801E0
:1023D00060913A024EE1E0DC682FCE0115DD1092EB
:1023E0000B020DC0E92FF0E0DE01AE0FBF1F149607
:1023F0008C91E45FFD4F80839F5F90930B029091DF
:102400000B02953078F302E580919703682F80FFE7
:10241000BBC081FF02C020E05FC09091210280918B
:102420000B02981799F5109221020EC0E22FF0E0EE
:10243000DF01A45FBD4FEE5DFD4F90818C91981739
:1024400049F42F5F209321022091210230910B0249
:10245000231760F32317D1F4809191039091920395
:10246000A0919303B09194032091360230913702EA
:102470004091380250913902821B930BA40BB50B8B
:102480008697A105B10510F421E001C020E010926B
:1024900021020CC0E92FF0E0DF01A45FBD4F8C9159
:1024A000EE5DFD4F80839F5F90932102909121020A
:1024B00080910B02981770F3809191039091920391
:1024C000A0919303B09194038093360290933702C6
:1024D000A0933802B09339020435F1F466FD1CC0B4
:1024E00080910B028530C0F080910E028B3409F48C
:1024F0004BC0893609F448C0833509F445C084359A
:1025000009F442C08D3709F43FC08E37E9F180915C
:102510000F0280778037C1F12223B1F5802F0E940E
:10252000B50680912002882329F080910B0281500A
:1025300080930B0210E008C0E12FF0E0E45FFD4F54
:1025400080810E943C071F5FE0910B021E17A0F3E1
:1025500080912002882359F0F0E0E45FFD4F8081F4
:1025600090E08F70907061E040E30E9407078091D7
:10257000970385FF05C084E30E940E030E943C0779
:102580000E94EA0601C000E08091970382FF6DC0BF
:1025900080E70E94B506888190E062E040E20E94F8
:1025A0004007888D90E014E0880F991F1A95E1F795
:1025B00065E040E20E944007898D90E0B4E0880F1A
:1025C000991FBA95E1F765E040E20E9440078A8DC5
:1025D00090E0A4E0880F991FAA95E1F765E040E23A
:1025E0000E9440078B8D90E0F4E0880F991FFA95C8
:1025F000E1F765E040E20E9440078A8190E063E0F5
:1026000040E20E944007898190E063E040E20E943E
:1026100040072B8187E090E0821B910962E040E255
:102620000E94400780E20E94B5068091970385FFD3
:1026300008C084E30E940E030E943C0780E20E94CF
:10264000B5068B81873019F089818F5F898310E00F
:1026500007C0FE01E10FF11D84810E943C071F5F4E
:1026600089811817B0F30E94EA06188280910A0245
:10267000815080930A02809109028F5F8093090242
:10268000843011F4109209027698043581F58CE0BB
:1026900092E00E945D1F2BC004E5B6CECE0165E43A
:1026A00023D9882309F04BCECE013ADA882311F0E2
:1026B00008E4AACECE011CDB882311F004E7A4CEE7
:1026C0008E01065E1F4FC80160913A024B8D64DB9C
:1026D000682FCE0199DBCE016BE406D9882309F47B
:1026E0005CCE47CE8981843009F04DCF64CEDF9136
:1026F000CF911F910F91089580919703882321F026
:102700000E9458040C9475030C943203FC018181DF
:10271000882371F4809197030E943C078091950370
:102720009091960365E040E20E9440070C94EA060F
:10273000CF01019667E973E041E00E947D07DCCF9D
:10274000A1E0B0E0E6EAF3E10C94CB2B8091240405
:10275000882309F484C0E0909103F09092030091E3
:10276000930310919403833009F060C08FE30E94BB
:102770000E03182F863010F400E018C08BEC94E0A4
:102780000E941A0928988FEF0E94080380E00E9497
:102790000803082F08C080E00E940803682F8BEC14
:1027A00094E00E941F091150B1F7289AA5DF1092FA
:1027B0002404053709F053C08EEC94E0BE016F5F2E
:1027C0007F4F41E00E947D07019759F599818091E3
:1027D0009D03981731F58091D204853539F00DC0ED
:1027E0008BEC94E00E9437090E94B5068091CD04DD
:1027F0008823B1F70E94EA0632C08091CD0484504C
:102800008093CD0484E08093CC048BEC94E06AE068
:102810000E941F09E0918D03F0918E0388E00995D5
:102820001EC08BEC94E00E941A0919C09E2D8230C4
:1028300049F480919C03981B983088F05DDF1092DA
:1028400024040DC0813059F487E390E00E9407040E
:102850000E94750382E080932404E0929C032196F9
:10286000E6E00C94E72B5B980C9436065B9A0C948C
:102870003606A7E0B0E0EFE3F4E10C94CA2B282F72
:102880008091A603843551F4809127049091280407
:102890000196909328048093270439C0863451F41C
:1028A00080912504909126040196909326048093AC
:1028B00025042DC0853451F480919A0390919B0397
:1028C000019690939B0380939A0321C08B3451F41B
:1028D00080912A0490912B04019690932B0480936D
:1028E0002A0415C0883451F480912C0490912D0451
:1028F000019690932D0480932C0409C08091980335
:10290000909199030196909399038093980385E79A
:102910008983222319F4DD24D39412C080912E04DC
:10292000BE016E5F7F4F0E94CF0780919D03BE0165
:102930006C5F7F4F0E94CF0785E58E8386E0D82E9F
:102940000E9458040E94860310E080E891E08EDF28
:1029500080E093E088DF1F5F1630B9F780E093E0F6
:1029600085DF80E891E07FDF80E891E07FDF5B98A2
:1029700087E390E00E94070483E00E943B062898CA
:102980008FE70E9408038091A0038D0D0E94080329
:102990007E010894E11CF11C8701F80181918F01EF
:1029A0000E940803802F8E198D15B8F306C08EE99A
:1029B00093E00E9437090E9408038091A0038823B6
:1029C000B1F7289A0E9486038EE993E00E941A09C3
:1029D00014E104C0115081E00E943B068AE30E948A
:1029E0000E0390E08F779070892B11F0112391F7EF
:1029F00083DE2796E7E00C94E62B82DB882361F0E8
:102A000083E080932904809121049091220401960F
:102A10009093220480932104809129048150809313
:102A20002904882321F083E080932304089581E022
:102A300020CFCF93DF93EC018981882339F48091F3
:102A40009D030E943C0780912E0413C08436A1F49C
:102A50008091910390919203A0919303B09194037C
:102A600064E040E30E9407078EE20E94B506809171
:102A700023040E943C074DC0833709F04DC080916C
:102A800027049091280461E040E30E9407078EE24A
:102A90000E94B506809125049091260461E040E3F0
:102AA0000E9407078EE20E94B50680919A039091DA
:102AB0009B0361E040E30E9407078EE20E94B50697
:102AC00080912A0490912B0461E040E30E94070763
:102AD0008EE20E94B50680912C0490912D0461E055
:102AE00040E30E9407078EE20E94B506809198039A
:102AF0009091990361E040E30E9407078EE20E94F3
:102B0000B506809121049091220461E040E30E9487
:102B100007070E94EA062CC08936D9F4CE01029636
:102B20006DE973E041E00E947D0780E690E06091EE
:102B30009D030E945508CE0104966EE274E041E0C8
:102B40000E947D0781E690E060912E040E94550866
:102B50000FC08EE993E00E941A0904C08EE993E049
:102B60000E941F09219668816623C1F780E081DEFB
:102B7000DF91CF91089580E690E00E94F107809365
:102B80009D0381E690E00E94F10780932E04882344
:102B900021F081E280939703AFCD0895A2E3B0E0E6
:102BA000E4EDF5E10C94CA2B80913C02882309F4F2
:102BB0009FC04A9B88C08FE30E940E038F778233A9
:102BC00068F08AE30E942A0386E30E942A038DE3C9
:102BD0000E942A0384E30E942A038AC089832898DA
:102BE0008FEF0E94080310E082E0E82EF12CEC0E3B
:102BF000FD1E08C080E00E940803F701E10FF11DEF
:102C000080831F5F89811817A8F380E00E94080362
:102C1000D82E80E00E940803289A84E30E942A03A9
:102C200085E30E940E038D30C1F79A8186E78927DC
:102C30008A8322E0AE014F5F5F4F08C0E40FF51FAB
:102C400080819452982790832F5F982F8981E22F5B
:102C5000F0E0281798F3E40FF51F80819B81892706
:102C600080838091970384FF13C081E60E94B5069C
:102C7000098110E07E010894E11CF11CF701E10FCD
:102C8000F11D80810E94B5061F5F0117B8F71BC0B8
:102C900081E40E94B506098110E07E010894E11CE0
:102CA000F11CF701E10FF11D80810E943C071F5FBD
:102CB0000117B8F78091970385FF03C08D2D0E94FF
:102CC0003C070E94EA0685E30E940E03813029F04A
:102CD000813161F48AE30E942A0386E30E942A0379
:102CE0008DE30E942A0384E30E942A030E94B60413
:102CF000E296E7E00C94E62BCF93DF93EA98209AD4
:102D0000289A8EE190E00E94360628988EE190E0A5
:102D10000E943606289A8DE290E00E94360680E3F3
:102D20000E942A0384E690E00E943606CCE7D2E0B7
:102D3000FE0184912196FE0164910E941C0321965C
:102D4000F2E0CE3ADF07A1F780913D02882371F0CF
:102D5000CEEAD2E0FE0184912196FE0164910E94A8
:102D60001C032196F2E0C43CDF07A1F783E30E9435
:102D70002A0384E00E943B0684E30E942A0385E341
:102D80000E940E038D30C1F7DF91CF910895A2E329
:102D9000B0E0EDECF6E10C94CA2B0196BE016F5F3A
:102DA0007F4F41E30E947D07D82E282F30E021502D
:102DB0003040898190E02817390709F072C080916E
:102DC0003C02882321F498DF83E00E943B061B81AC
:102DD0008A8196E789278A8322E0AE014F5F5F4FA1
:102DE0000BC0FA01EA0FFB1FAC0FBD1F8C91845280
:102DF0009081892780832F5F8981A22FB0E02817D7
:102E000080F3FA01EA0FFB1F80818127808385E32D
:102E10000E942A0385E30E940E038331C1F714FF49
:102E200008C088E70E943B0688E70E943B0688E7C7
:102E300001C08AE00E943B0628988FE70E940803A1
:102E40007E010894E11CF11C870105C0F801819105
:102E50008F010E940803802F8E198D15B8F3289AD0
:102E600085E30E940E038331D9F385E30E940E03AC
:102E7000863149F48BE30E942A0386E30E942A03E9
:102E80008DE30E942A0380913C02882349F084E369
:102E90000E942A0385E30E940E038D30C1F701C012
:102EA0002BDCE296E7E00C94E62BFC0101962181F5
:102EB000223731F0223559F481E080933D0202C07F
:102EC00010923D0219DF81E080933C020895233780
:102ED00009F45DCF10923C0208951F93CF93DF93C6
:102EE000EA98209A289A8EE190E00E943606289867
:102EF0008EE190E00E943606289A8DE290E00E94D2
:102F0000360680E30E942A0384E690E00E9436069B
:102F1000C4ECD2E0FE018491813450F42196FE018C
:102F200064910E941C032196F3E0C030DF0791F703
:102F300083E30E942A0384E00E943B0610E01150C4
:102F400041F084E30E942A038AE090E00E94360662
:102F5000F6CF81E080933E02DF91CF911F910895DB
:102F6000EF92FF920F931F93CF93DF937C01EB01BE
:102F7000FC0100810F5F6115710519F420E030E05C
:102F800002C024E630E0802F90E043E0880F991FD4
:102F90004A95E1F76AE070E00E94AC2B260F371FDC
:102FA000A901662757FD6095762F209195033091F2
:102FB0009603C901A0E0B0E084179507A607B707FC
:102FC00028F489E093E00E94EE06CEC0241B350B66
:102FD000309396032093950380913E02882309F451
:102FE0007CDF85E30E940E038D3071F08AE50E943C
:102FF000B50685E40E94B50682E50E94B50682E525
:103000000E94B50681E34AC0809145029091460234
:10301000A0914702B09148020097A105B10521F4A3
:1030200029C081E00E943B06809191039091920318
:10303000A0919303B09194032091450230914602F0
:10304000409147025091480282179307A407B507A1
:1030500041F38091910390919203A0919303B091D9
:1030600094032F5F3F4F4F4F5F4F82179307A40783
:10307000B507B9F20E94860385E30E940E038331EF
:10308000C1F08AE50E94B50685E40E94B50682E596
:103090000E94B50682E50E94B50682E30E94B5064D
:1030A00085E30E940E030E943C070E94EA0615DF9A
:1030B0005BC0CD2B49F0C0E0D0E084E60E943B0627
:1030C0002196CA30D105C9F728988FE70E940803D6
:1030D000E70110E004C089910E9408031F5F1017E8
:1030E000D0F3289A10E085E30E940E038D3059F04A
:1030F00085E30E940E03833131F481E00E943B0698
:103100001F5F183C81F785E30E940E038D30B9F0F4
:103110008AE50E94B50685E40E94B50682E50E9414
:10312000B50682E50E94B50683E30E94B50685E3F5
:103130000E940E030E943C070E94EA06CEDE8091A8
:103140003E02882309F4D8DA80919103909192038A
:10315000A0919303B091940380934502909346020B
:10316000A0934702B0934802CDB7DEB7E6E00C94D7
:10317000E72BEF92FF920F93DF93CF93CDB7DEB79C
:103180002C970FB6F894DEBF0FBECDBFFC018BE0CD
:10319000898381818A831B8282E08C8387818D83EE
:1031A00080858E8381858F838481888785818987C7
:1031B00086818A871B861C8684E10E943B067E01ED
:1031C0000894E11CF11CC70160E070E0C9DE8AE5EB
:1031D0000E94B50600E006C0EE0DFF1D80810E9432
:1031E0003C070F5FE02FF0E0898190E08E179F078A
:1031F0009CF78091970385FF03C080E00E943C0705
:103200000E94EA062C960FB6F894DEBF0FBECDBF23
:10321000CF91DF910F91FF90EF900895CF93DF93BF
:10322000EC0190913F02992341F480914002882360
:1032300021F4809141028823B1F48B81803321F005
:10324000803411F0803579F48F81891761F4988585
:1032500080914002981739F499858091410298171E
:1032600011F4CE0186DF90914202992341F48091BE
:103270004302882321F4809144028823A9F08881A5
:103280008B3091F48B81803479F48F81891761F4CC
:10329000988580914302981739F49985809144026A
:1032A000981711F4CE0165DFDF91CF910895AEE15B
:1032B000B0E0EDE5F9E10C94CB2B80913E02882340
:1032C00009F46AC04A9B5AC08FE30E940E038F77AD
:1032D00089838E3110F08DE1898328988FEF0E94C9
:1032E000080310E052E0E52EF12CEC0EFD1E08C0A4
:1032F00080E00E940803F701E10FF11D80831F5F4A
:1033000089811817A8F380E00E940803082F80E045
:103310000E940803289A7E010894E11CF11CC70151
:103320007DDF8091970384FF10C08AE70E94B50675
:1033300010E007C0F701E10FF11D80810E94B50682
:103340001F5F89818117B0F727C08AE50E94B50603
:1033500010E007C0F701E10FF11D80810E943C07DA
:103360001F5F89818117B0F78091970385FF03C0A4
:10337000802F0E943C070E94EA060EC085E30E944F
:103380000E03813149F48AE30E942A0386E30E94F6
:103390002A0384E30E942A036E96E6E00C94E72B4E
:1033A000AEE1B0E0E6EDF9E10C94CD2B8C01FC012F
:1033B0008181823711F491DD37C0833711F0863671
:1033C00001F5C8010296BE016F5F7F4F4DE10E947B
:1033D0007D0790E00197298130E08217930729F05B
:1033E00080E093E00E94EE061FC060E070E0F8010C
:1033F0008181833711F461E070E0CE010196B0DD88
:1034000013C0813629F4C80102966FE372E006C04A
:10341000873741F4C801029662E472E043E00E94FB
:103420007D0702C010923E026E96E4E00C94E92BF8
:10343000AEE1B0E0EEE1FAE10C94CA2B80914902D2
:10344000882309F476C04A9B61C08FE30E940E0373
:103450008F7789838E3110F08DE1898328988FEFE3
:103460000E94080310E082E0E82EF12CEC0EFD1E15
:1034700008C080E00E940803F701E10FF11D80837E
:103480001F5F09811017A8F380E00E940803D82E5F
:10349000289A8AE30E942A0386E30E942A038DE386
:1034A0000E942A0384E30E942A038091970384FFE9
:1034B00012C087E70E94B50610E07E010894E11C67
:1034C000F11CF701E10FF11D80810E94B5061F5F1D
:1034D0000117B8F72EC087E50E94B50610E07E01FF
:1034E0000894E11CF11CF701E10FF11D80810E949D
:1034F0003C071F5F0117B8F78091970385FF03C052
:103500008D2D0E943C070E94EA0613C085E30E94AD
:103510000E03813011F0813161F48AE30E942A03A5
:1035200086E30E942A038DE30E942A0384E30E941B
:103530002A036E96E7E00C94E62BCF93DF93EA988C
:10354000209A289A8EE190E00E94360628988EE113
:1035500090E00E943606289A8DE290E00E9436069E
:1035600080E30E942A0384E690E00E943606C9E1C7
:10357000D3E0FE018491813450F42196FE016491E0
:103580000E941C032196F3E0C535DF0791F783E322
:103590000E942A0381E00E943B06DF91CF910895AB
:1035A000FC018181823729F4C8DF81E080934902E0
:1035B0000895833711F0109249020895282F813021
:1035C00091F45B9A20910B0130910C01C901880F95
:1035D000991F820F931F0E9436065B9880910B0102
:1035E00090910C0134C080910B0190910C01222329
:1035F00009F55B9A0E9436065B9820910B01309189
:103600000C01C901880F991F820F931F0E94360673
:103610005B9A80910B0190910C010E9436065B9899
:1036200020910B0130910C01C901880F991F820F65
:10363000931F20C05B9A0E9436065B9820910B0175
:1036400030910C01C901880F991F820F931F0E94AE
:1036500036065B9A20910B0130910C01C901880F4D
:10366000991F820F931F0E9436065B9880910B0171
:1036700090910C010C9436060F931F93CF93DF9318
:10368000EA98209A289A8EE190E00E9436062898BF
:103690008EE190E00E943606289A8DE290E00E942A
:1036A000360680E30E942A0384E690E00E943606F4
:1036B000289880E40E940803C5E5D3E0FE018491C8
:1036C0000E9408032196F3E0C236DF07B9F7809124
:1036D0000F010E940803809110010E94080380914D
:1036E00011010E9408032396FE0184910E940803A1
:1036F0002196F3E0CE37DF07B9F7289A28988EE7AE
:103700000E9408038BE290E08C010F5F1F4F0E9424
:10371000F1070E940803C80103331105A9F7289A8D
:1037200083E30E942A0381E00E943B0681E08093AC
:103730008F03DF91CF911F910F910895CF92DF9268
:10374000EF92FF921F93CF93DF937C01FC01818165
:10375000843759F4C70102966BE071E00E94B0070C
:1037600080910B0190910C0111C0833709F0A5C025
:10377000F7018281823789F4C70103966DE071E019
:103780000E94B00780910D0190910E0160E040E22F
:103790000E9440070E94EA06FBC0769A80914C0284
:1037A0008823B1F480913C02882329F081E0809342
:1037B0004A0210923C0280913E02882329F081E067
:1037C00080934B0210923E0257DF83E00E943B063B
:1037D00086E30E942A038AE30E942A038BE30E9465
:1037E0002A030E948603CC24DD2424C08A818033EE
:1037F00011F480E005C0813311F481E001C082E062
:10380000DDDE1F5F21961D3089F75B9A80910B01E9
:1038100090910C010E9436065B9810E080910B019C
:1038200090910C010E9436061F5F1F31B9F7089472
:10383000C11CD11C80910D0190910E01C816D906B2
:1038400018F4E70111E0D2CF80914C02882341F0B7
:1038500080919703882371F486E30E942A0317C09E
:1038600080914A02882349F010924A0245DA81E0A9
:1038700080933C020E9475030AC080914B0288230A
:1038800021F010924B0229DB02C00E947C13769833
:1038900089E60E94B50683E70E94B506E70111E0BC
:1038A0008A81803319F0813309F086E40E94B506DD
:1038B0001F5F21961D30A1F76DCF8237B9F480913B
:1038C0003C02882329F081E080934A0210923C0256
:1038D00080913E02882329F081E080934B02109270
:1038E0003E02CADE81E080934C0252C0863659F512
:1038F000F7018281803351F480E180930F0180EBE6
:103900008093100181E78093110107C0C7010296DF
:103910006FE071E043E00E947D0789E60E94B506F2
:1039200086E60E94B5068AE30E94B50680910F01E3
:103930000E943C07809110010E943C078091110178
:103940000E943C0727CF883719F580914A028823C7
:1039500039F010924A02D0D981E080933C0210C025
:1039600080914B02882321F010924B02B6DA0EC0F0
:1039700082E090E00E94070480919703882319F069
:103980000E94750303C086E30E942A0310924C0232
:10399000DF91CF911F91FF90EF90DF90CF9008952E
:1039A0002F923F924F925F926F927F929F92AF922F
:1039B000BF92CF92DF92EF92FF920F931F93DF930C
:1039C000CF930F92CDB7DEB77C01FC0181818337A5
:1039D00009F075C1198287E090E00E94F62B6C0116
:1039E000C70102968E010F5F1F4FB80141E00E9490
:1039F0007D078981F60181935F01C7010496B801B3
:103A000041E00E947D078981807FF6018183C701A3
:103A10000696B80141E00E947D078981F601828304
:103A2000C7010896B80141E00E947D078981F6012F
:103A30008383C7010A96B80141E00E947D0789810E
:103A4000F6018683C7010C96B80141E00E947D070C
:103A50008981F6018583C7010E96B80141E00E9475
:103A60007D078981F60184833181160120E057E0CA
:103A7000452E512C4C0C5D1C9191892F82958F7095
:103A800089272827E415F505B9F72F70232BF501B1
:103A90002083F60196012A5F3F4F8181908189271B
:103AA00081833196E217F307C1F7769A80914F022E
:103AB000882309F059C080913C02882329F081E0D5
:103AC00080934D0210923C0280913E02882329F09F
:103AD00081E080934E0210923E02EA98209A289A42
:103AE0008EE190E00E94360628988EE190E00E94D8
:103AF0003606289A8DE290E00E94360680E30E9406
:103B00002A0384E690E00E943606289880E40E940A
:103B100008030EE713E0F80184910E9408030F5F89
:103B20001F4FF3E0073A1F07B1F7289A28988EE74E
:103B30000E9408038BE290E08C010F5F1F4F0E94F0
:103B4000F1070E940803C80103331105A9F7289A59
:103B500083E30E942A0381E00E943B0681E0809378
:103B60008F0383E00E943B0686E30E942A038AE3D8
:103B70000E942A038BE30E942A030E9486035B9A19
:103B800087EC94E20E9436065B9889E50E943B062A
:103B900085E392E00E943606AA24BB2456C0AA20E0
:103BA00011F402E001C007E010E05B9A86EF99E0B3
:103BB0000E9436065B9886EF99E00E9436061F5FEA
:103BC00010179CF35B9A8CEF92E10E9436065B988B
:103BD00080911501909116010E9436068601F80128
:103BE000808140E8E42EF12C9924682E7724C701C7
:103BF000862197212091150130911601892B31F4EE
:103C00005B9AC9010E9436065B9805C05B98C901A2
:103C10000E9436065B9A80911501909116010E94D0
:103C200036069394F8E09F1619F0F694E794DFCFE8
:103C30000F5F1F4F0415150591F65B9880E090E02B
:103C40000E9436060894A11CB11C8091120190E0DC
:103C5000A816B9060CF4A3CF80914F02882341F037
:103C600080919703882371F486E30E942A0317C08A
:103C700080914D02882349F010924D023DD881E099
:103C800080933C020E9475030AC080914E028823F3
:103C900021F010924E0221D902C00E947C13769826
:103CA00089E50E94B50683E70E94B506F10181917E
:103CB0001F010E943C0724143504C1F718C0823745
:103CC000C9F4C701029662E171E00E94B00789E57C
:103CD0000E94B50682E70E94B5068AE30E94B506F7
:103CE0008091120190E060E040E20E9440070E9453
:103CF000EA0652C0843751F5F7018281803339F4E6
:103D000088ED94E0909314018093130106C0C701DD
:103D1000029663E171E00E94B007809113019091D7
:103D2000140196958795909316018093150189E566
:103D30000E94B50684E70E94B5068AE30E94B50694
:103D4000809113019091140166E0CECF883721F560
:103D500080914D02882341F010924D020E947C1602
:103D600081E080933C0210C080914E02882321F0B4
:103D700010924E02B2D80EC082E090E00E9407047A
:103D800080919703882319F00E94750303C086E38E
:103D90000E942A0310924F020F90CF91DF911F9142
:103DA0000F91FF90EF90DF90CF90BF90AF909F90DA
:103DB0007F906F905F904F903F902F900895DC011F
:103DC000E8E5F2E00EC0109751F091818C919817C0
:103DD00031F4928111968C9111979817A1F0E20F0E
:103DE000F11D2081222321F083E0E630F80758F30B
:103DF00083E0E630F80719F010F0E6E0F3E0AB2BD3
:103E000011F0E0E0F0E0CF010895CF93DF93EC01F3
:103E1000D6DFFC01009779F0909106038081981716
:103E200050F4E90FF11D80818A8389E78B838181BA
:103E30008C8381E001C080E0DF91CF9108950F93E2
:103E40001F93CF93DF938C018091970386FF18C057
:103E500084E50E94B506C0E0D0E0F801EC0FFD1F3C
:103E600080810E943C072196C530D105B1F7809131
:103E7000970385FF03C08AEF0E943C070E94EA0671
:103E8000DF91CF911F910F91089586E30E942A033D
:103E900080915302833511F08BE401C08BE90E94BD
:103EA0003B0681E592E065E04CE021E00E94920B48
:103EB0000E94750381E592E0C2CF1F93FC0140810F
:103EC00031811281938124818FE580934604109281
:103ED000570250912F04552329F4809145048823DB
:103EE00009F4CDC080915102841721F480915202CF
:103EF000831771F0109231041092500283E0809386
:103F000006038FEF80934604409351023093520290
:103F1000809131048F3F09F4B2C010935302909303
:103F20005402209355021123E1F08823D1F4251780
:103F300061F0243651F0812F8355823010F01D3707
:103F400021F48FEF809331049AC0143509F497C09F
:103F5000892F807F803609F092C090679093540239
:103F600083C081E592E051DF882329F480913104F8
:103F7000882309F484C090915002992311F0892F6D
:103F800006C0E0913104F0E0E955FC4F849183359F
:103F900041F4143531F4809131048E5F8093310403
:103FA0000BC0811749F0109231041092500283E047
:103FB000809306038FEF61C0992379F08091060307
:103FC0008E5F8093060381E592E01FDF882371F402
:103FD000809131048E5F8093310490913104E92FF8
:103FE000F0E0E855FC4F14911F3F59F480915302C3
:103FF000809350028436C1F580913004809355023D
:1040000033C01093530287E78093540280912F04AA
:1040100080935502892F8E5F809331041092500255
:104020008E3001F581E592E0CADEFC01009781F057
:10403000808190E026E033E0281B390BDF01A80FD8
:10404000B91F02C08D918193E217F307D8F3108254
:10405000109231041092500283E0809306038FEF98
:1040600080934604112359F010DF80915302893662
:1040700031F081E08093570289E2809346041F91DA
:10408000089580915702882351F0FFDE89E28093E2
:1040900046048091570281508093570208951092F0
:1040A00031041092500283E0809306038FEF8093D7
:1040B00046040895A6E0B0E0E0E6F0E20C94C92BD7
:1040C0004091450480913204882341F0833019F0F7
:1040D0008DE790E015C087E791E012C0842F90E053
:1040E000877090702DE730E0BC01629FC001639F34
:1040F000900D729F900D1124825B9F489595879536
:1041000090933404809333044A831B8205E314E0C4
:10411000FF246E010894C11CD11C8CE2E82EF8012A
:1041200090819F3FB1F080912F048F0D8983809102
:104130003204882311F0EC8203C09C83F801818152
:104140008D83C60165E04CE021E00E94920BC60120
:1041500076DEF3940E5F1F4FF8E0FF1601F78091B3
:104160003204882341F0833019F41092320403C0E2
:104170008250809332042696E8E00C94E52B85E388
:1041800090E00E94F10780932F0486E390E00E9464
:10419000F10780934504E5E3F4E09FEF90833296C6
:1041A00084E0E534F807D1F7109231041092500200
:1041B00083E080930603909346041092580208957A
:1041C0006F927F929F92AF92BF92CF92DF92EF92C7
:1041D000FF920F931F93DF93CF9300D000D000D0B6
:1041E000CDB7DEB73C017C010894E11CF11CC7018E
:1041F000BE016F5F7F4F45E00E947D07E9818430FB
:1042000008F0ADC0E130A9F4833061F485E390E0BB
:104210006A810E94550886E390E06B810E945508F0
:10422000AEDF23C180912F040E943C07809145049A
:1042300091C0E23009F04DC0813029F020E030E03B
:104240008A81813011F421E030E0E22E8091580221
:10425000882321F48FEB93E00E94EE0608E512E03C
:104260002EC082E00835180719F080E20E94B506DA
:10427000F80181810E943C07F80182810E943C077D
:10428000EE20C9F08AE30E94B50653E0F52E0FC078
:10429000F3E0FF1528F4F0FE03C08CE20E94B5069F
:1042A000F801EF0DF11DF39480810E943C07F801A5
:1042B0008081F81668F3F8018081080F111DF8015C
:1042C0008081882309F448C0F3E006301F0748F2D4
:1042D00043C0E33049F480E090E071DD28E532E04E
:1042E0002255281B822F36C0E03149F505E314E042
:1042F000EE24FF24F80180818F3FA1F0EE2019F019
:1043000080E20E94B5068F2D0E943C078AE30E943E
:10431000B506F80180810E943C07F80181810E9466
:104320003C07E3940E5F1F4FF394F8E0FF1611F77C
:10433000EE2091F48BEB93E00E94EE060DC0E1318C
:1043400059F480913304909134046DE770E00E9439
:10435000982B862F0E943C070E94EA0686C0809117
:104360002F04E817D0F1482F50E0F0E0CA0107967B
:104370008E179F0794F19A8180914504981769F5EB
:104380008C818F3231F4C3016CE042E00E94070C53
:104390006CC02D818C32C1F42093320481E090E016
:1043A000909334048093330430E0220F331F220FA4
:1043B000331F8091950390919603820F931F9093E2
:1043C00096038093950351C0E41BF50BEE0FF0E0CC
:1043D000EB5CFB4F8083218348C080E090E0EFDC02
:1043E0008C01D7010D900020E9F71197AE19BF0994
:1043F000B695A7959A2E9394890D911D8855924054
:104400008F3A910574F5F80190827801DD24D394F8
:10441000CC24C3941BC057010894A11CB11CC30138
:104420008C0D911DB50141E00E947D07F2E0FD1564
:1044300048F4D0FC07C0F7018081843619F48181EB
:1044400080933004F2E0CF0ED3947501D91418F3A1
:1044500083E00630180748F40D0D111DF801108295
:1044600004C085EB93E00E94EE0626960FB6F89402
:10447000DEBF0FBECDBFCF91DF911F910F91FF9097
:10448000EF90DF90CF90BF90AF909F907F906F9014
:104490000895A0E8B0E0EFE4F2E20C94C92B80911B
:1044A0004704882309F455C0813011F580919103A8
:1044B00090919203A0919303B091940320910703EC
:1044C000281709F446C085E30E940E03813129F4C0
:1044D0008AE30E942A030E947503809191039091C0
:1044E0009203A0919303B09194038093070331C08A
:1044F0008FE30E940E03D82E87FD28C028988FEFE7
:104500000E9408037E010894E11CF11C8701CE2C57
:1045100006C080E00E940803F80181938F01802F7C
:104520008C198D15B0F3289A81E08093930105C012
:10453000F70181917F010E94B5068E2D8C198D1592
:10454000B8F30E94EA068FEF8093930181E0809395
:104550004704C058DF4FE8E00C94E52B0F931F93FE
:10456000CF93DF93EC01DC010D900020E9F7119768
:10457000A81BB90B8981823751F487E390E00E9430
:1045800007040E94750381E08093470429C08337A4
:1045900029F50A2F28988FE70E940803802F825060
:1045A0000E94080312E004C089810E9408031F5F73
:1045B00021961017C8F3289A0E94860304C084E647
:1045C00090E00E9436068AE30E940E0390E08F7707
:1045D0009070892BA1F70E94750302C010924704C6
:1045E000DF91CF911F910F9108950F931F93CF9358
:1045F000DF93EC0100E0802F90E09C01220F331F3D
:10460000280F391FF901E455FF4F1491F901E355C3
:10461000FF4F25913491112399F0209739F480E2CE
:104620000E94B506812F0E94B50608C088818117B7
:1046300029F4CE01F901099581E003C00F5FDBCFBA
:1046400080E0DF91CF911F910F9108951F931091FA
:1046500093018093930135C08BEC94E00E9437095D
:104660008A3011F08D3009F5E0910803EE2349F10D
:10467000F0E0E75FFC4F108289E093E0B6DF88232B
:1046800089F48BED93E00E94EE0689E093E00E94AE
:10469000FB0683EC93E00E94EE0680E090E0A5DF4D
:1046A0000E94EA06109208030CC09091080397FD3F
:1046B00008C0E92FF0E0E75FFC4F80839F5F909395
:1046C00008038091CD04882339F6109393011F913C
:1046D0000895E4E6F0E080818B7F8083299A84B19D
:1046E000876084B9239880E58CBD8DB581608DBDD0
:1046F00008954091D2085091D3084115510521F4F5
:104700004091890150918A0120918B0130918C0157
:104710002115310541F42DB73EB780918701909165
:104720008801281B390B4217530718F020E030E0AE
:1047300002C0241B350BC901089582E40E94B5060E
:104740008091D2089091D30865E040E20E94400732
:104750000E94EA0683E50E94B50680918901909146
:104760008A0165E040E20E9440070E94EA0685E473
:104770000E94B50680918B0190918C0165E040E22A
:104780000E9440070E94EA0686E40E94B506B1DF57
:1047900065E040E20E9440070C94EA06A2E0B0E027
:1047A000E3EDF3E2FCC7E3E5F5E08091F1008193EE
:1047B00085E0EB35F807C9F7809153053091540532
:1047C000353009F49FC0363048F4313009F44BC01D
:1047D000313070F0333009F023C145C0383009F46E
:1047E000D7C0393009F4FCC0363009F019C1B4C063
:1047F000803821F0823809F013C108C090914E052D
:1048000080914F05882391F0926010C080915705E8
:104810008093E9008091EB0090E025E096958795E4
:104820002A95E1F7982F91701092E9008091E800A5
:10483000877F8093E8009093F1001092F1008091BF
:10484000E800982F9E7F9093E8008F778093E80090
:1048500005C080915205882309F4E4C08091E800E6
:1048600082FFF7CFB3C0882319F0823009F0D8C097
:1048700090E08F719070009719F00297B9F50CC015
:1048800080915505813009F0CDC010924F0533302D
:1048900069F580934F052AC080915505882331F52D
:1048A00020915705277009F4BDC02093E90080913D
:1048B000EB0080FF1BC03130A1F48091EB008061E0
:1048C0008093EB0081E090E002C0880F991F2A9549
:1048D000E2F78093EA001092EA008091EB00886092
:1048E00003C08091EB0080628093EB001092E9009E
:1048F0008091E800877F8093E8008091E800982FFE
:104900009E7F68C0882309F08BC020915505809157
:10491000E800877F8093E8008091E800982F9E7FD1
:104920009093E8008F778093E80005C0809152054E
:10493000882309F477C08091E80080FFF7CF922F99
:104940009F77892F80688093E300992309F46AC0D8
:1049500083E08093520566C08058823008F060C0C2
:10496000809155059091560560915705AE014F5FB6
:104970005F4F0E94C802BC01009709F453C08091A8
:10498000E800877F8093E80089819A812AD11EC040
:10499000803809F045C08091E800877F8093E80067
:1049A000809150058093F1008091E800982F9E7FC0
:1049B0009093E8008F778093E80004C080915205BF
:1049C000882381F18091E80082FFF8CF8091E80090
:1049D000982F9B7F9093E8008F778093E80022C008
:1049E0008823F1F4209155052230E0F48091E8000D
:1049F000877F8093E800209350058091E800982FEE
:104A00009E7F9093E8008F778093E800222311F037
:104A100084E001C083E0809352050E94720502C0C9
:104A20000E9434058091E80083FF0AC08091EB006A
:104A300080628093EB008091E800877F8093E8009C
:104A40002296E2E0C8C68093E9008091EB00816085
:104A50008093EB001092ED006093EC004093ED002A
:104A60008091EE00881F8827881F08951092F40017
:104A700090E09093E9001092F0001092E80080918D
:104A8000ED008D7F8093ED008091EB008E7F809311
:104A9000EB009F5F973069F7089580915305882355
:104AA000BCF404C0809152058823F9F08091E8009D
:104AB00082FFF8CF8091E800982F9B7F9093E800C9
:104AC0008F778093E800089580915205882369F0DC
:104AD0008091E80080FFF8CF8091E800982F9E7FBA
:104AE0009093E8008F778093E800089594E6809192
:104AF000EC0080FF05C08091E80080FF05C01FC06A
:104B00008091E80082FD1BC080915205882311F43A
:104B100082E008958091EB0085FF02C081E0089556
:104B20008091E10082FFE3CF8091E1008B7F809351
:104B3000E100992311F483E008959150D8CF80E0EB
:104B40000895FC014091590550915A059B01461763
:104B5000570708F49A0140E032C08091E80083FFD3
:104B600002C081E008958091E80082FD32C080910A
:104B700052058823A1F18091E80080FF20C005C084
:104B800081918093F100215030402115310531F0A1
:104B90008091F2009091F300089790F38091F200D9
:104BA0009091F30040E0089709F441E08091E8001B
:104BB000982F9E7F9093E8008F778093E8002115CF
:104BC000310559F6442349F604C0809152058823E3
:104BD00031F08091E80082FFF8CF80E0089582E014
:104BE0000895DC014091590550915A059B014617E3
:104BF000570708F49A0140E034C08091E80083FF31
:104C000002C081E008958091E80082FD34C0809167
:104C100052058823B1F18091E80080FF22C007C0CF
:104C2000FD011196E491E093F100215030402115EF
:104C3000310531F08091F2009091F300089780F3F4
:104C40008091F2009091F30040E0089709F441E070
:104C50008091E800982F9E7F9093E8008F77809353
:104C6000E8002115310549F6442339F604C0809146
:104C70005205882331F08091E80082FFF8CF80E070
:104C8000089582E00895FC0124C08091E80083FF2C
:104C900002C081E0089580915205882341F18091FE
:104CA000E80082FFF2CF06C08091F100819361504D
:104CB000704031F08091F2009091F300892BA1F7C0
:104CC0008091E800982F9B7F9093E8008F778093E6
:104CD000E80061157105C9F604C08091520588236A
:104CE00031F08091E80080FFF8CF80E0089582E005
:104CF000089567D06ED01092520510925005109210
:104D00004F0510924E058AE482BF19BC89B58260B6
:104D100089BD09B400FEFDCF8091D800982F9F7700
:104D20009093D80080688093D8008091D7008160EC
:104D30008093D7008091D8008F7D8093D800809198
:104D4000E0008B7F8093E0008091E0008E7F809375
:104D5000E0008091E1008E7F8093E1008091E2008D
:104D600081608093E2008091E100877F8093E10081
:104D70008091E20088608093E2008091D800816099
:104D80008093D8000895B5DFE0EEF0E08081816087
:104D90008083E8EDF0E080818F77808319BC80818B
:104DA0008F7E8083109251050895A3DFE8EDF0E037
:104DB00080818061808381E080935105789408959B
:104DC0000895E8EDF0E080818E7F80831092E2000C
:104DD00008951092DA001092E10008951F920F9248
:104DE0000FB60F9211242F933F934F935F936F93BE
:104DF0007F938F939F93AF93BF93EF93FF93809194
:104E0000DA0080FF15C08091D80080FF11C080912A
:104E1000DA008E7F8093DA008091D90080FF05C090
:104E200081E080935205CCDF03C010925205C8DFA9
:104E30008091E10080FF1DC08091E20080FF19C0D9
:104E40008091E1008E7F8093E1008091E2008E7F6F
:104E50008093E2008091E20080618093E200809183
:104E6000D80080628093D80019BC85E080935205F9
:104E7000A7DF8091E10084FF29C08091E20084FFD8
:104E800025C019BC89B5826089BD09B400FEFDCF7B
:104E90008091D8008F7D8093D8008091E1008F7E33
:104EA0008093E1008091E2008F7E8093E200809108
:104EB000E20081608093E20080915005882311F424
:104EC00083E001C084E0809352057ADF8091E100A5
:104ED00083FF23C08091E20083FF1FC08091E10027
:104EE000877F8093E10082E0809352051092500505
:104EF0008091E1008E7F8093E1008091E2008E7FBF
:104F00008093E2008091E20080618093E200AEDD58
:104F100080E060E042E097DD53DFFF91EF91BF91C9
:104F2000AF919F918F917F916F915F914F913F9141
:104F30002F910F900FBE0F901F9018951F93809187
:104F40005205882361F01091E9001092E9008091E8
:104F5000E80083FF01C022DC17701093E9001F9165
:104F600008951F93CF93DF93182F53985298109260
:104F70008A03EA98209A289A8EE190E00E943606E9
:104F800028988EE190E00E943606289A8DE290E003
:104F90000E94360680E30E942A0384E690E00E9485
:104FA0003606113019F0123089F511C0CFEDD3E07B
:104FB000FE0184918134D8F42196FE0164910E940F
:104FC0001C032196F4E0C73ADF0791F710C0CCE24A
:104FD000D4E0FE018491813450F42196FE01649165
:104FE0000E941C032196F4E0C43FDF0791F7109361
:104FF0008A0383E30E942A038CE0EEE7F6E0DF01F8
:105000001D928A95E9F784E00E943B06DF91CF91DB
:105010001F910895FC018181823771F48281882378
:1050200069F0833711F481E003C0843719F482E01A
:1050300098DF04C080E0FCCF833799F080918A0329
:10504000813019F0823039F403C083E894E005C060
:105050008DE794E002C089E794E00E94EE060C948C
:10506000EA060895FF920F931F93CF93DF93182FB3
:10507000092FF62E28988FEF0E940803212F302F3A
:10508000C901EC0110E005C080E00E94080389938B
:105090001F5F1F15C8F3289ACDB7DEB7E5E098C3A8
:1050A0001F93882339F485E30E940E038D3011F499
:1050B00080E03EC01092890686E30E942A0385E3C1
:1050C0000E940E03182F8130D1F78BE30E942A0330
:1050D0008AE30E942A0310927E06109280061092A4
:1050E0007F0610928206109281068AE896E09093DD
:1050F000840680938306109285061093860610928C
:10510000870680918A038093880683E060E00E948E
:105110001C0388E062E00E941C0384E30E942A03CF
:1051200085E30E940E038D30D9F781E080938906D4
:105130001F910895A2E0B0E0EFE9F8E22FC380915B
:105140008A03882309F4ECC080918906813051F0EC
:10515000813030F0823061F0833009F09DC06FC043
:1051600081E0DDC04A9B98C082E08093890694C0AC
:105170004B9B92C0809183069091840663E072DF1E
:10518000809188062091830630918406BE016F5F6E
:105190007F4F813061F4C901C6D0882309F0BBC0BC
:1051A000898180937E067CD1AC0181E00CC0C9016D
:1051B00040E008D1882309F0AEC0898180937E0643
:1051C0006FD1AC0180E060E083D190938006809342
:1051D0007F0660917F067091800682E069347807CF
:1051E00008F099C06F3F710509F058F486E00E94FD
:1051F0001C0388E060E00E941C0381E08093850628
:1052000003C086E00E941C0380918306909184066F
:105210000396909384068093830680917F069091F5
:1052200080060397909382068093810610928606EB
:1052300083E08093890667E00E941C032DC04B9B8E
:105240002BC080918106909182068F3F910509F0D5
:1052500058F480918506882339F488E060E00E9444
:105260001C0381E0809385068091830690918406DB
:105270006FE1F8DE80918106909182064F979093BE
:1052800082068093810680918306909184064F96D2
:1052900090938406809383064A9940C08091890642
:1052A000823008F43BC0809183069091840660911F
:1052B0008106D8DE81E08093870680918806813060
:1052C00051F480917E06ECD0AC018AE896E06BE563
:1052D00075E0A2D109C080917E06E2D0AC018AE8D7
:1052E00096E06BE575E00FD1892BA9F482E60E9468
:1052F000B50610E006C0E55AFA4F80810E943C07CF
:105300001F5F80915B05CCD0E12FF0E0E817F90733
:1053100090F30E94EA061092890602C080E0C0DE87
:105320002296E3E057C2CF93DF93FC01EB01A0810B
:105330008181EA2FE295EF70F0E0E95EFE4F508147
:10534000B0E0AF70B070A95EBE4FAC91E82FE295AF
:10535000EF70F0E0E95EFE4F4081E82FF0E0EF7083
:10536000F070E95EFE4FE08120E030E0EF3F11F4A5
:1053700021E030E080E090E04F3F11F481E090E0E8
:10538000282B392B80E05F3F09F481E090E0AF3FAC
:1053900009F491E0892B90E0282B392B232B11F075
:1053A00081E00DC05295550F550F507CA295A07FFE
:1053B000A52BAE2B440F440F4A2B488380E0DF918E
:1053C000CF9108950F931F93CF93DF93EC018B013F
:1053D000442319F050E060E01AC08A81E82FF0E021
:1053E000EF73F070E95CFE4F6081E981F0E0EF70EF
:1053F000F070EE0FFF1FEE0FFF1F829586958695CA
:10540000837090E0E82BF92BE95CFE4F5081A88176
:10541000E981E295EF70F0E08A2F90E08370907060
:1054200024E0880F991F2A95E1F7E82BF92BE95C16
:10543000FE4FE081A695A695B0E0A95CBE4FAC9169
:1054400020E030E0EF3F11F421E030E080E090E038
:10545000AF3F11F481E090E0282B392B80E06F3FC3
:1054600009F481E090E05F3F09F491E0892B90E03E
:10547000282B392B232B11F081E00DC0A295A07FA2
:10548000AE2BF801A083442329F45295507F562B6C
:10549000F801518380E0DF91CF911F910F91089522
:1054A000482F8A3110F422E009C090E04A9754E076
:1054B000959587955A95E1F7282F2D5F842F90E0D9
:1054C000019630E0220F331F280F391FC9010895BC
:1054D000882351F0662321F09A012F5F3F4F01C0CE
:1054E0009A01220F331F0DC09A01220F331F240F80
:1054F000351F36952795662311F440FF02C02F5FB4
:105500003F4FC9010895A0E0B0E0E8E8FAE23FC1EA
:105510005C018B017A01CC24DD24C0E0D0E06BC0BB
:1055200081E0E816F10491F4C501B80141E04ADFD9
:10553000882309F067C0C095D095D070F8018081AC
:1055400090E0C817D90709F45AC05FC0C501B80177
:1055500040E038DF882309F055C08EEF9FEFE80E5A
:10556000F91EE2E0F0E0CE0EDF1EE114F10459F086
:10557000FBE0CF16D104E0F0C6010C9762E170E0C9
:10558000D7D0892BA9F4AE01409550959A0130707F
:10559000F801818190E028173907B9F5252F3327C5
:1055A000808190E02817390781F5C0E0D0E01DC068
:1055B000F1E0EF16F10489F4CE01F80160819DD08D
:1055C000EC019C0120953095232F3327F801818130
:1055D00090E02817390749F018C0CE01F801608122
:1055E0008CD0F801618189D0EC0183E090E0A80EB5
:1055F000B91E0E5F1F4FE114F10409F091CF20E0B6
:1056000030E005C021E030E002C022E030E0C90116
:10561000CDB7DEB7EAE0D7C0A0E0B0E0E1E1FBE261
:10562000B2C03C016B014A01AA24BB24C0E0D0E017
:1056300000E010E0EE24FF2452C0C301B60173DE87
:10564000882319F021E030E053C082E088169104ED
:1056500069F09AE0A916B10458F000E010E0C50125
:105660000A9762E170E064D0892B11F401E010E048
:10567000E114F10471F0C095D095D070F6018081ED
:1056800090E0C817D90791F5C0E0D0E0EE24FF24E0
:1056900019C00115110589F09E0120953095232F21
:1056A0003327F601808190E028173907F9F400E0EC
:1056B00010E041E0E42EF12C05C0CE01F60160813E
:1056C0001CD0EC010894810891080894A11CB11C1D
:1056D00082E090E0680E791E0894C11CD11C8114F0
:1056E000910409F0AACF20E030E002C022E030E0CF
:1056F000C901CDB7DEB7EEE062C0AC0170E0E5E60F
:10570000FDE39A0120703078232F3327862F90E015
:1057100080789070440F551F2817390711F04E27D5
:105720005F277F5F783011F0660FEBCFCA010895D5
:10573000AA1BBB1B51E107C0AA1FBB1FA617B707B7
:1057400010F0A61BB70B881F991F5A95A9F78095D3
:105750009095BC01CD01089597FB092E07260AD02C
:1057600077FD04D0E5DF06D000201AF4709561952E
:105770007F4F0895F6F7909581959F4F08952F924A
:105780003F924F925F926F927F928F929F92AF92D1
:10579000BF92CF92DF92EF92FF920F931F93CF931E
:1057A000DF93CDB7DEB7CA1BDB0B0FB6F894DEBFB5
:1057B0000FBECDBF09942A88398848885F846E84DB
:1057C0007D848C849B84AA84B984C884DF80EE8025
:1057D000FD800C811B81AA81B981CE0FD11D0FB62E
:1057E000F894DEBF0FBECDBFED010895CF93DF93D8
:1057F000BC018230910510F462E070E0A091D40801
:10580000B091D508ED01E0E0F0E040E050E021C0CB
:10581000888199818617970769F48A819B813097DF
:1058200019F09383828304C09093D5088093D408A1
:10583000FE0134C06817790738F44115510519F095
:105840008417950708F4AC01FE018A819B819C01B5
:10585000E9012097E9F641155105A9F1CA01861B16
:10586000970B049708F4BA01E0E0F0E02AC08D91AC
:105870009C91119784179507F9F46417750781F4C3
:1058800012968D919C911397309719F09383828390
:1058900004C09093D5088093D408FD0132964FC080
:1058A000CA01861B970BFD01E80FF91F61937193E5
:1058B00002978D939C9343C0FD01828193819C014B
:1058C000D9011097A1F68091D2089091D308892B25
:1058D00041F48091890190918A019093D30880933B
:1058E000D20840918B0150918C014115510541F432
:1058F0004DB75EB78091870190918801481B590B85
:105900002091D2083091D30824173507B0F4CA018A
:10591000821B930B8617970780F0AB014E5F5F4F9A
:105920008417950750F0420F531F5093D3084093AC
:10593000D208F9016193719302C0E0E0F0E0CF0179
:10594000DF91CF910895CF93DF93009709F450C072
:10595000EC0122971B821A82A091D408B091D5083D
:10596000109709F140E050E0AC17BD0708F1BB8388
:10597000AA83FE0121913191E20FF31FAE17BF07F9
:1059800079F48D919C911197280F391F2E5F3F4F0D
:105990003983288312968D919C9113979B838A83D8
:1059A0004115510571F4D093D508C093D40820C097
:1059B00012968D919C911397AD01009711F0DC0127
:1059C000D3CFFA01D383C28321913191E20FF31F28
:1059D000CE17DF0769F488819981280F391F2E5F60
:1059E0003F4FFA01318320838A819B819383828395
:1059F000DF91CF910895F999FECF92BD81BDF89ABC
:105A0000992780B50895262FF999FECF1FBA92BD28
:105A100081BD20BD0FB6F894FA9AF99A0FBE01968F
:065A20000895F894FFCF89
:105A26008025000000000802323100A401060010A3
:105A3600B07106D8046C02FFFFFFFFFF0302FFFFF1
:105A46000100FFFFFFFFFFAAA9A6A59A9996956AEE
:105A56006966655A595655FFFFFFFFFFFFFFFFFFB7
:105A6600FFFF03FF0102FFFFFFFF07FFFF00FFFF2E
:105A76000506FF04FFFFFFFFFFFF0BFF090AFFFFFD
:105A86000FFFFF08FFFFFFFF0D0EFF0CFFFFFFFFDD
:105A9600FFFFFFFFFFFFFF160D0E0B1C191A132C3D
:0E5AA600252623343132292000D608000000C6
:00000001FF
